:1000000000C001206D000000910000009100000080
:10001000910000009100000091000000000000002D
:10002000000000000000000000000000910000003F
:10003000910000000000000091000000910000000D
:100040009100000000F000B806480749097800F068
:1000500001F8FEE703781BB18B4202D00130F9E7CB
:100060000020704700000020050000200549064AD6
:10007000064B9A42BEBF51F8040B42F8040BF8E756
:10008000FFF7E0FF940000000000002008000020BF
:04009000FEE700BFC8
:0800940048656C6C007100006E
:040000030000006D8C
:00000001FF
